:100000000C9462010C948A010C948A010C948A016C
:100010000C948A010C948A010C948A010C948A0134
:100020000C948A010C948A010C947F060C944B0565
:100030000C948A010C948A010C948A010C948A0114
:100040000C948A010C948A010C948A010C948A0104
:100050000C948A010C948A010C948A010C94A401DA
:100060000C948A010C948A010C948A010C948A01E4
:100070000C948A010C948A010C948A010C948A01D4
:100080000C948A010C948A010C948A010C948A01C4
:100090000C948A010C948A010C948A010C948A01B4
:1000A0000C948A010C948A010C948A01A702AA027A
:1000B00099029D02A302CB02CB02CB02AE02B20296
:1000C000B602BC02C002CB02C60200000002000958
:1000D0000F0000030401000C00000408020110409E
:1000E000804010204080408008020401010210205E
:1000F00040801080102040400404040404030405E0
:1001000002020202040302020202060606060606B4
:1001100004040202020400000000250028002B0055
:100120002E00310000000000240027002A002D00CE
:10013000300000C18081C112010002020000408D28
:100140000E01AB00010102000112010002000000DB
:10015000408D0E01AB0001010200014D6564696133
:1001600054656B204C616273004C696E6B4974205E
:10017000536D61727420373638380004030904085F
:100180000B0002020201000904000001020200004B
:1001900005240010010524010101042402060524A0
:1001A0000600010705810310004009040100020A4E
:1001B000000000070502024000000705830240001E
:1001C0000000000000000000002A2B2800000000B2
:1001D000000000000000000000000000000000001F
:1001E000002C9EB4A0A1A2A434A6A7A5AE362D379C
:1001F00038271E1F20212223242526B333B62EB7ED
:10020000B89F8485868788898A8B8C8D8E8F909104
:1002100092939495969798999A9B9C9D2F3130A391
:10022000AD350405060708090A0B0C0D0E0F101159
:1002300012131415161718191A1B1C1DAFB1B0B5DF
:10024000000904020001030000000921010100016E
:100250002265000705840340000105010902A10190
:100260000901A100850105091901290315002501CE
:10027000950375018102950175058103050109301A
:10028000093109381581257F750895038106C0C09D
:1002900005010906A1018502050719E029E71500F6
:1002A0002501750195088102950175088103950660
:1002B0007508150025650507190029658100C0002E
:1002C000B107040911241FBECFEFDAE0DEBFCDBFB6
:1002D00011E0A0E0B1E0E2E8F2E102C005900D9289
:1002E000A832B107D9F721E0A8E2B1E001C01D9220
:1002F000A739B207E1F712E0C4ECD2E004C02297BC
:10030000FE010E943B09C03CD107C9F70E943C0393
:100310000C943F090C94000061E08DE00C94CC0239
:1003200061E08DE00E94050364E670E080E090E00B
:100330000E94110260E08DE00E94050364E670E017
:1003400080E090E00C9411021F920F920FB60F9272
:1003500011242F933F938F939F93AF93BF938091DB
:10036000290190912A01A0912B01B0912C0130918B
:10037000280126E0230F2D3720F40296A11DB11D80
:1003800005C029E8230F0396A11DB11D2093280164
:100390008093290190932A01A0932B01B0932C0103
:1003A00080912D0190912E01A0912F01B0913001EB
:1003B0000196A11DB11D80932D0190932E01A09354
:1003C0002F01B0933001BF91AF919F918F913F91D9
:1003D0002F910F900FBE0F901F9018953FB7F89474
:1003E00080912D0190912E01A0912F01B0913001AB
:1003F00026B5A89B05C02F3F19F00196A11DB11D80
:100400003FBF6627782F892F9A2F620F711D811D9C
:10041000911D43E0660F771F881F991F4A95D1F7FA
:100420000895CF92DF92EF92FF92CF93DF936B010B
:100430007C010E94EE01EB01C114D104E104F1043E
:1004400089F00E94F3060E94EE016C1B7D0B683E52
:10045000734090F381E0C81AD108E108F108C8514F
:10046000DC4FEACFDF91CF91FF90EF90DF90CF90FC
:100470000895789484B5826084BD84B5816084BD1C
:1004800085B5826085BD85B5816085BDEEE6F0E00D
:10049000808181608083E1E8F0E010828081826069
:1004A0008083808181608083E0E8F0E080818160EA
:1004B0008083E1E9F0E080818260808380818160D7
:1004C0008083E0E9F0E0808181608083E1ECF0E00E
:1004D000808184608083808182608083808181606C
:1004E0008083E3ECF0E0808181608083E0ECF0E0E9
:1004F000808182608083E2ECF0E080818160808393
:10050000EAE7F0E08081846080838081826080837C
:1005100080818E7F8083808180688083089590E0D1
:10052000FC013197EF30F105B0F5EA5AFF4F0C941A
:100530003909809180008F7703C0809180008F7D82
:1005400080938000089580918000877FF9CF84B5E3
:100550008F7702C084B58F7D84BD0895809190000F
:100560008F7707C0809190008F7D03C080919000AD
:10057000877F8093900008958091C0008F7703C09B
:100580008091C0008F7D8093C00008958091C2004B
:10059000877F8093C2000895CF93DF9390E0FC01A2
:1005A000E652FF4F2491FC01E850FF4F84918823CD
:1005B00049F190E0880F991FFC01EC5DFE4FA59179
:1005C000B4918A5E9E4FFC01C591D4919FB7611191
:1005D00008C0F8948C91209582238C938881822383
:1005E0000AC0623051F4F8948C91322F30958323F5
:1005F0008C938881822B888304C0F8948C91822B01
:100600008C939FBFDF91CF9108950F931F93CF934A
:10061000DF931F92CDB7DEB7282F30E0F901E65304
:10062000FF4F8491F901E652FF4F1491F901E85010
:10063000FF4F04910023C9F0882321F069830E94B1
:100640008F026981E02FF0E0EE0FFF1FEA5EFE4FA0
:10065000A591B4919FB7F8948C91611103C0109546
:10066000812301C0812B8C939FBF0F90DF91CF918D
:100670001F910F91089508950E9439020E943B0333
:1006800081E391E00E94D5060E948C01C0E0D0E099
:100690000E9490012097E1F30E940000F9CF409161
:1006A00035015091360120913301309134014217C8
:1006B0005307B4F49091E8009570E1F39091E8004D
:1006C00092FD19C08093F10080913501909136011F
:1006D00001968F739927892B19F48EEF8093E80088
:1006E0008091350190913601019690933601809367
:1006F000350181E0089580E00895CF92DF92FF9266
:100700000F931F93CF93DF931F92CDB7DEB7082FC0
:10071000162F862F880F8E5F99830E944F0383E0E8
:100720000E944F03F02EC02E9981D92E8C2D8F1947
:10073000811778F4F60184910E944F03082F80E01E
:100740000E944F038023FFEFCF1ADF0A8111EECF03
:1007500001C081E00F90DF91CF911F910F91FF9029
:10076000DF90CF900895615030F02091F100FC01AE
:1007700020830196F8CF289884E680933801089565
:100780002FB7FC012083F89467706093E900089507
:10079000CF93DF931F92CDB7DEB7682FCE010196BE
:1007A0000E94C0038091F20099819FBF0F90DF915A
:1007B000CF910895FF920F931F93CF93DF9300D0B3
:1007C000CDB7DEB7F62E8A0190913701992311F04B
:1007D00057FF03C08FEF9FEF2BC0682FCE0101960C
:1007E0007A830E94C0038091F20090E0A8017A8190
:1007F000801791070CF4AC01EF2DF72FF40E84E66F
:10080000FE1639F02898809338019091F100919369
:10081000F7CF4115510521F08091F200882321F096
:1008200089818FBFCA0104C08BE68093E800F8CFAE
:100830000F900F90DF91CF911F910F91FF9008952E
:10084000CF93DF931F92CDB7DEB741E050E0BE01FA
:100850006F5F7F4F0E94DA03019719F4898190E05E
:1008600002C08FEF9FEF0F90DF91CF910895CF934C
:10087000DF931F92CDB7DEB7682FCE0101960E949D
:10088000C0039091E800892F807295FF04C0909179
:10089000F20080E4891B99819FBF0F90DF91CF9177
:1008A00008956F927F928F929F92AF92BF92CF9254
:1008B000DF92EF92FF920F931F93CF93DF931F92DC
:1008C000CDB7DEB7782E7B01C42EB52E80913701CF
:1008D000882369F0042F152F8AEFD82E872D807278
:1008E000982E9AE3A92E872D8074882E11C08FEF41
:1008F0009FEF57C0872D0E943704682E81110CC0CE
:10090000DA94A9F361E070E080E090E00E941102C7
:100910000115110579F73BC0282F30E002171307A6
:100920000CF4602E672DCE0101960E94C0038091C9
:10093000E80085FF29C0262D30E0021B130B99200B
:1009400039F06A948FEF6816B1F01092F100F9CF88
:10095000F701862D77FE07C0815058F0949190934F
:10096000F1003196F9CF815020F091919093F100F0
:10097000FACFE20EF31E8091E80085FF0FC001154B
:10098000110511F481100AC089818FBFC1CF5D9814
:1009900084E6809339018C2D9B2D03C0A092E80042
:1009A000F3CF0F90DF91CF911F910F91FF90EF90B8
:1009B000DF90CF90BF90AF909F908F907F906F907F
:1009C00008951092E900109236011092350190932B
:1009D0003401809333010895CF92DF92FF920F93F9
:1009E0001F93CF93DF9300D0CDB7DEB7F82E8A01E7
:1009F0006B0101151105B1F0F601F7FE02C08491FB
:100A000001C0808149835A830E944F03015011091C
:100A1000FFEFCF1ADF0A49815A818111EACF8FEFA8
:100A20009FEF01C0CA010F900F90DF91CF911F91EE
:100A30000F91FF90DF90CF9008951F93CF93DF9396
:100A40001F92CDB7DEB7162F2091E80022FFFCCF12
:100A5000612F79830E94B3038BEF8093E800812F8D
:100A60007981972F0F90DF91CF911F910895CF93A8
:100A7000DF931F92CDB7DEB71982CE0101960E9497
:100A80005107CE0101960E94EC07898190E00F90FA
:100A9000DF91CF9108951F920F920FB60F921124FC
:100AA000EF92FF920F931F932F933F934F935F9378
:100AB0006F937F938F939F93AF93BF93EF93FF9326
:100AC000CF93DF93CDB7DEB76297DEBFCDBF109275
:100AD000E9008091E80083FFEBC068E0CE010A9650
:100AE0000E94B30382EF8093E8009A8597FF05C0C8
:100AF0008091E80080FFFCCF03C08EEF8093E80078
:100B0000892F807609F0B9C08B85811105C01092BC
:100B1000F1001092F100C5C0282F2D7F213009F47B
:100B2000C0C0853049F48091E80080FFFCCF8C85FF
:100B300080688093E300B5C0863009F076C02D85CB
:100B4000E888F988223071F580E090E02A8B0E94D5
:100B5000E1040E94370599E08E010F5F1F4FF801F5
:100B6000392F11923A95E9F799832A892A8391E0DE
:100B70009E8390E898879AEF99872091350130916C
:100B80003601275F3F4F3C832B838D83C7010E9433
:100B9000E10449E050E0B80180E00E94EC040E94CA
:100BA00037057FC0C7012A8B0E94E1042A892232BF
:100BB00041F482E290E00E94F707892B09F071C0AE
:100BC00074C0213069F488899989089711F42093B9
:100BD000320180913201811118C069E471E01AC0BC
:100BE000233009F062C08C85882391F0823021F493
:100BF00061E189E691E006C0813009F056C06DE000
:100C00008BE591E00E947D034AC067E371E002C07A
:100C10006BE771E06115710509F447C0FB01449170
:100C200050E080E80E94EC043CC0873009F43DC0ED
:100C3000883021F481E08093F10033C0893089F558
:100C4000937099F5E3E3F1E081E021E096E380938E
:100C5000E9002093EB0034913093EC009093ED0089
:100C60008F5F3196853099F78EE78093EA00109276
:100C7000EA008C858093370114C0888999890E9485
:100C8000E1048E85811105C0CE010A960E945C07A1
:100C900006C0823051F4CE010A960E941F088823B4
:100CA00021F08EEF8093E80003C081E28093EB0097
:100CB00062960FB6F894DEBF0FBECDBFDF91CF9125
:100CC000FF91EF91BF91AF919F918F917F916F9124
:100CD0005F914F913F912F911F910F91FF90EF9056
:100CE0000F900FBE0F901F9018958093E900809190
:100CF000F200882319F08AE38093E80008951F9298
:100D00000F920FB60F9211242F933F934F935F933F
:100D10006F937F938F939F93AF93BF93EF93FF93C3
:100D20008091E1001092E10083FF0FC01092E90072
:100D300091E09093EB001092EC0092E39093ED0021
:100D40001092370198E09093F00082FF1DC083E07D
:100D50000E94750680913901882339F0809139010C
:100D6000815080933901882369F08091380188236C
:100D700059F080913801815080933801811104C06D
:100D8000289A02C05D9AF1CFFF91EF91BF91AF9188
:100D90009F918F917F916F915F914F913F912F9193
:100DA0000F900FBE0F901F9018951092370181E0A1
:100DB0008093D70080EA8093D80082E089BD09B48F
:100DC00000FEFDCF61E070E080E090E00E94110243
:100DD00080E98093D8008CE08093E2001092E000DC
:100DE000559A209A08950895CF93DF931F92CDB717
:100DF000DEB76983DC01ED91FC910280F381E02D87
:100E000041E050E0BE016F5F7F4F09950F90DF9189
:100E1000CF910895CF93DF93EC018C859D8597FF4B
:100E200005C082E00E9420049D878C878C859D856B
:100E3000DF91CF91089583E00C947506FC018485C1
:100E4000958597FD06C082E00E94C80390E0019658
:100E5000089582E00E94C80390E00895FC01848513
:100E6000958597FD05C02FEF3FEF358724870895BF
:100E700082E00C942004CF93DF93EC018091070172
:100E8000882331F083E00E9451041816190634F0CB
:100E900081E090E09B838A8380E090E0DF91CF91B6
:100EA0000895FC0120812E5F208342E450E06FE72B
:100EB00071E080E80C94EC04FC0181819081913A0E
:100EC00059F4813209F03CC047E050E060E071E045
:100ED00080E00E94EC0443C0913291F5803239F4F5
:100EE00067E070E080E091E00E941D0506C082325C
:100EF00009F035C0828180930701809100019091B3
:100F00000101A0910201B0910301803B9440A10531
:100F1000B105C1F48091070180FD14C087E797E710
:100F200090930108809300082BE088E190E00FB6D1
:100F3000F894A895809360000FBE209360000FC0C6
:100F400080E0089588E10FB6F894809360001092D5
:100F500060000FBEA895109201081092000881E071
:100F6000089510923D0110923C0188EE93E0A0E0BC
:100F7000B0E080933E0190933F01A0934001B09375
:100F800041018EE091E090933B0180933A018FEF15
:100F90009FEF90934701809346010895FF920F932E
:100FA0001F93CF93DF93EC01F62EE881F981048043
:100FB000F581E02D09958C01E881F9810680F781A2
:100FC000E02D6F2DCE010995C8019927DF91CF91B2
:100FD0001F910F91FF900895FC0120812F5F2083C6
:100FE00049E150E061E472E080E80C94EC0445E6ED
:100FF00050E06AE572E080E80C94EC04EF92FF9216
:101000000F931F93CF93DF931F92CDB7DEB78983E2
:101010008B017A0141E050E0BE016F5F7F4F84E0B9
:101020000E945104A701B80184E40E9451040F906A
:10103000DF91CF911F910F91FF90EF900895FC01E8
:1010400091818081813A31F481E0913091F0933047
:1010500089F411C0813271F49B3021F48281809334
:10106000090105C09A3031F482818093080181E042
:101070000895089580E0089548E050E082E00C94DF
:10108000FE07CF93DF93DC01683818F0E8E7E60F3E
:1010900025C0E62FF0E067FF11C0E058F10981E0BC
:1010A00090E001C0880FEA95EAF714969C91149796
:1010B000982B14969C931497E0E010C0EF53FE4FCA
:1010C000E491EE2309F440C0E7FF08C014968C9128
:1010D0001497826014968C931497EF7716968C91E0
:1010E00016978E1741F117968C9117978E1719F155
:1010F00018968C9118978E17F1F019968C91199774
:101100008E17C9F01A968C911A978E17A1F01B961C
:101110008C911B978E1779F080E090E0ED01C80F5D
:10112000D91F2E81211102C0EE8305C001968630A1
:101130009105A1F709C0BD016C5F7F4FCD010E94F1
:101140003C0881E090E008C081E090E013969C9319
:101150008E93129780E090E0DF91CF9108956838E8
:1011600018F0E8E7E60F25C0E62FF0E067FF12C0B1
:10117000E058F10921E030E001C0220FEA95EAF7DA
:101180002095DC0114963C911497322314963C93DD
:10119000E0E00FC0EF53FE4FE491EE2329F1E7FFAB
:1011A00008C0DC0114962C9114972D7F14962C9373
:1011B000EF7720E030E0EE2351F0DC01A20FB31F07
:1011C00016964C9116974E1302C016961C922F5FDE
:1011D0003F4F2630310579F7BC016C5F7F4F0E948D
:1011E0003C0881E090E0089580E090E00895FC01E3
:1011F0001682178210861186128613861482BC010D
:101200006C5F7F4F0C943C081092960110928D01F8
:1012100010928C018EE191E090938B0180938A0172
:101220000895CF92DF92EF92FF920F931F93CF9387
:10123000DF936C017A01EB01E60EF71E00E010E08F
:10124000CE15DF0561F06991D601ED91FC91019019
:10125000F081E02DC6010995080F191FF1CFC801D3
:10126000DF91CF911F910F91FF90EF90DF90CF9082
:101270000895EE0FFF1F0590F491E02D0994F89466
:02128000FFCF9E
:1012820000E1000000000000010100000000F4067F
:101292003B071E072E070A071B0700000000CE07A8
:0812A20011094108AF08F7082B
:00000001FF
